:1000000006C2000021C200001FC200000C94400F75
:100010001BC2000019C2000017C200000C942F0F71
:1000200013C2000011C200000FC200000DC2000088
:100030000BC2000009C2000007C2000005C2000098
:1000400003C2000001C20000FFC10000FDC10000AA
:100050000C94C20EF9C10000F7C10000F5C1000008
:10006000F3C10000F1C10000EFC10000EDC10000CC
:10007000EBC10000E9C10000E7C1000032303232BC
:10008000303831373037313400FF07FF07AE042AEC
:100090000530068C06A5069B067E065606EE06A7CC
:1000A000065F069C064D06670616061C061706C662
:1000B00005B805A4058C0570055105310533050DFE
:1000C00005E804DE04B704A80480046D0446043285
:1000D000040B04F503DF03BA03A40381036B034A93
:1000E0000334031603F802DB02C002A60286026E86
:1000F00002510236021602FE01DE01C401A7018987
:10010000016C01520136011801FF00FF00FF00FFE2
:1001100000FF00FF00FF00FF00FF00FF00FF00FFE7
:1001200000FF00FF00FF00FF00FF00FF00FF00FFD7
:1001300000FF00FF00FF00FF00FF00FF00FF00FFC7
:1001400000FF00FF00FF00FF00FF00FF00FF00FFB7
:1001500000FF00FF00FF00FF00FF00FF00FF00FFA7
:1001600000FF00FF00FF00FF00FF00FF00FF00FF97
:1001700000FF00FF00FF00FF00FF00FF00FF00FF87
:1001800000FF00FF00FF00FF00FF00FF00FF00FF77
:1001900000FF00FF00FF00FF00FF00FF00FF00FF67
:1001A00000FF00FF00FF00FF00FF00FF00FF00FF57
:1001B00000FF00FF00000000000000000000000041
:1001C000000000000000000000000000000000002F
:1001D000000000000000000000000000000000001F
:1001E000000000000000000000000000000000000F
:1001F00000000000000000000000000000000000FF
:1002000000000000000000000000000000000000EE
:1002100000000000000000000000000000000000DE
:1002200000000000000000000000000000000000CE
:1002300000000000000000000000000000000000BE
:1002400000000000000000000000000000000000AE
:10025000000000000000000000000000000000009E
:100260000000000000000000000100030004000680
:1002700000070009000B000C000E00100012001413
:1002800000160018001B001D001F0022002500277B
:10029000002A002D0030003300360039003D0040B8
:1002A00000440048004B004F00530058005C0061C0
:1002B0000065006A006F00740079007E0084008A87
:1002C00000900096009C00A200A900B000B700BEFC
:1002D00000C500CD00D500DD00E500ED00F600FF13
:1002E00000010003000300040005000600070008E9
:1002F0000009000A000C000D000E00100011001390
:100300000014001600180019001B001D001F00211A
:10031000002300250028002A002C002F0031003483
:1003200000360039003B003E0040004300460048D4
:10033000004B004D00500052005500570059005B23
:10034000005D005F0060006200630064006400659F
:100350000064006400630061005F005D005A0056A5
:1003600000520057005B00600064006A006F007478
:10037000007A00800086008D0093009B00A200A9F7
:1003800000B100BA00C200CB00D500DE00E800F3E7
:1003900000FE00FF00FF00FF00FF00FF00FF00FF66
:1003A00000FF00FF00FF00FF00FF00FF00FF00FF55
:1003B00000FF00FF00FF00FF00FF00FF00FF00FF45
:1003C00000FF00FF00FF00FF00FF00FF00FF00FF35
:1003D00000FF00FF00FF00FF00FF00FF00FF00FF25
:1003E00000FF00FF00FF00FF00FF00FF00FF00FF15
:1003F00000FF00FF00FF00FF00FF00FF00FF00FF05
:1004000000FF00FF00FF00FF00FF000000001124BC
:100410001FBECFEFCDBFDFE3DEBF18E3A0E0B8E340
:10042000E6E3F5E202C005900D92A032B107D9F7DC
:1004300028E3A0E2B8E301C01D92A93CB207E1F7AE
:100440000E94500F0C948E12DBCDF89498ED94BF5F
:10045000809361008091630080FDFCCF78940895C3
:10046000E6E9F8E320E030E09081992339F02F5F4E
:100470003F4F339620313105B9F70BC0F901EE0F2C
:10048000FF1F2E0F3F1FF901EA56F74C808361834F
:10049000728308950F931F93CF93DF93D091963873
:1004A000DD2351F10091973810919838C09173383D
:1004B000C150C7FD0DC0EC2FEE0FFF0BEC58F74CF1
:1004C0000190F081E02DB8018D2F09958111F0CFB9
:1004D000E6E9F8E383818083848195818183928337
:1004E000339688E3E33CF807A9F71092C3381092DB
:1004F000C4381092C538D2CFDF91CF911F910F91A0
:100500000895BC018091C838ABCF1092C8381092C2
:10051000C6381092C73881E080934D3808950F9304
:100520001F93CF93C82F02E919E0CC2349F085E04F
:100530008CDFC8010197F1F781E087DFC150F5CF6B
:10054000CF911F910F910895E0E0F6E082858160E0
:100550008287808581608087089582B185FB8827A6
:1005600080F991E0892780936C380895E0910638EE
:10057000F09107383196FB70F460E0930638F09301
:100580000738809168388B5A80936838E49180915D
:1005900068388E0F0895882349F0813069F480E22D
:1005A0008093220488E080933504089580E280934C
:1005B000210480932604089580E28093210480938F
:1005C00025040895CF93C82F80936A3880936938A3
:1005D00080916B38811101C0DEDFC11109C010921A
:1005E0003A0A10923B0A1092380A1092390A24C033
:1005F0008FEF8C0F90E0880F991FFC01EF51FD4F9A
:100600002591349120933A0A30933B0AFC01EB5434
:10061000FE4F259134912093380A3093390AFC011A
:10062000E757FF4F859194918093360A9093370A4C
:1006300080912938811104C01092200A1092210A59
:10064000C0932938C23010F485E001C081E0CF9119
:10065000FCCECF93DF93CDB7DEB72697CDBFDEBFFD
:1006600090914838209184383091853821503B4012
:1006700009F492E0843019F4609349381FC066236E
:10068000E9F0823019F427E9261B622F26E0E0E228
:10069000F5EADE01119601900D922A95E1F79E018F
:1006A0002F5F3F4F280F311D280F311DF901329761
:1006B0000190F081E02DE90FF11D60832696CDBFFA
:1006C000DEBFDF91CF910895BF92CF92DF92EF927C
:1006D000FF920F931F93CF93DF93EC014091483823
:1006E000E0911A38EE2311F082E001C0842F90E0EF
:1006F000DC01AC5EB74C2C9120931838DC01AF5E66
:10070000B74C8C9180931738F0E0E25FF74C318161
:10071000622F70E0442349F0313039F49B01280FF7
:10072000311DC9019595879538C0C617D707A4F123
:10073000682F70E06C177D0784F1411102C08C2F87
:100740002CC0821B032F10E001501109E82EF12C60
:10075000C701B8010E944712609346386695E62F9C
:10076000F0E0822FC12CD12CB12CB316B1F0C60110
:10077000B8010E943312822F860FCE0CDF1CAE010F
:10078000481B510957FF03C0519541955109E41782
:10079000F5071CF4B394E9CF822FDF91CF911F911D
:1007A0000F91FF90EF90DF90CF90BF9008958093CE
:1007B0004C3808CFCF93C0916A3889E18C0F8739C4
:1007C00008F080E0FFDE82E0AADE8C2FCF91FACE27
:1007D000CF93C0916A3880E0F5DE83E0A0DE8C2FF5
:1007E000CF91F0CE81E00895611160931D38089596
:1007F000662389F0813061F4809187389091863842
:10080000891B681B6093863882E080931E3803C082
:10081000635E60931C3880911C38873418F086E43E
:1008200080931C3808956093413808950F931F9367
:10083000CF93DF938091483880934E38809114385D
:1008400080934F38809111388093503880910E38C2
:1008500080935138809115388093523880911238A6
:100860008093533880910F38809354388091163894
:100870008093553880911338809356388091103882
:100880008093573880911A3880935838809149382E
:10089000809359388091473880935A38809119381D
:1008A00080935B3880914B3880935C3880914A38D4
:1008B00080935D3880910B3880935E388091093841
:1008C00080935F3880910A3880936038809108382F
:1008D0008093613880910C388093623880911C3805
:1008E00080936338809186388093643880911D3876
:1008F0008093653880910D388093663880914138B7
:1009000080936738F8940EE418E3C1E4D0E0F8016E
:1009100061918F01CE010E9471122196CB35D105D4
:10092000B1F765EA80E490E00E9471127894DF915B
:10093000CF911F910F9108951092953890911006C4
:1009400080916838890F8093683880918A3888232D
:1009500009F419C110928A389091933880916B38BC
:10096000882339F0809100068E7F809300061092D4
:100970009338911143C080911E38882349F06091CB
:100980008F387091903860938B3870938C3804C096
:1009900060918B3870918C38605F7F4FA6E07695C0
:1009A0006795AA95E1F780E098E50E94331280915F
:1009B0001D3890E00297680F791F769567956093D0
:1009C000893880913D38882311F0815007C06D31FE
:1009D00038F460E070E084E043DD85E080933D38EA
:1009E00080916B388111C6C08EE18093060685E444
:1009F0008093020681E080939338B9C0913009F06A
:100A0000B9C080911E38811143C080918D3890917A
:100A10008E3840969C0145E0369527954A95E1F73A
:100A2000A0918638A901569547950A2E000CBB0B5C
:100A3000CD0183519140840F951F80938738909307
:100A4000883880912C38E82FF0E0EE0FFF1FE35D2F
:100A5000F74C40815181B901641B750B20833183B0
:100A60008F5F877080932C38CB01880F991F880F78
:100A7000991F40911C3850E04D5E5E4F4A1B5B0B46
:100A8000440F551F841B950B820F931F23E01CC03E
:100A9000809191389091923880938D3890938E38D0
:100AA000409635E0969587953A95E1F7EDE2F8E3C3
:100AB0008193919328E3ED33F207D1F7A6CF009706
:100AC00009F00196215029F018161906C4F701976C
:100AD000F9CF18161906E4F477FD39C020912B38A8
:100AE00012160CF1880F991FBC016350710977FF32
:100AF00002C06F5F7F4F759567951616170614F045
:100B000061E070E088E1861B80932B3885E026C089
:100B10008C3F2FEF9207DCF477FF19C020912B3820
:100B200027FF05C02450281B20932B3818C024EE23
:100B3000281B20932B38209189382F3180F06CEFBF
:100B40007FEF681B790B7595679586E007C08091EC
:100B500089388E3120F060E070E087E081DC8DE143
:100B60008093060685E580930206109293381092D2
:100B70009438EADC80911E38882329F080911E3851
:100B8000815080931E380895813019F410924B38AB
:100B90000895823019F460934A380895833019F427
:100BA000609347380895843011F46093193808959C
:100BB000909189389D3110F480E009C083708330B2
:100BC00039F46F70E62FF0E0EA5DFA458081E3CCFE
:100BD0000895CF93C0911A38C1114AC0883039F4B2
:100BE00010924538109242381092433842C0813BEF
:100BF00059F48091453881508330D0F583E080935B
:100C000045388093443834C0853BB1F4CB016EE362
:100C100070E00E943312892B61F5809145388A3F3C
:100C200040F58B5F8093453880934438109242386A
:100C300010924338BFDD1DC08130D1F4809142381D
:100C400090914338019688382EE0920728F48093DB
:100C50004238909343380DC0109242381092433876
:100C600080914538882329F081508093453801C010
:100C7000C1E08C2FCF910895FF920F931F93CF93D4
:100C8000DF938C01EB01F42E8091843890918538AC
:100C9000892B31F0E0918438F091853889E009950D
:100CA0000093843810938538012B39F0E091843813
:100CB000F0918538BE018F2D099581E080934D38E4
:100CC000DF91CF911F910F91FF900895CF93DF9304
:100CD000E0917338EE2359F0E150E0937338F0E07F
:100CE000EE0FFF1FEC58F74CC081D18102C0C0E06D
:100CF000D0E0E0917338EE2341F0F0E0EE0FFF1FFB
:100D0000EE58F74C8081918102C080E090E04AE08B
:100D100060E070E0B1DFCE01DF91CF9108958830BF
:100D200029F410923E381092243815C08130F9F41D
:100D300090912438911107C06032710568F1809359
:100D40002438E3DB29C0913081F46B3B710528F036
:100D500082E08093243880E01EC061157105E1F0C7
:100D60006270862F880F8E5E16C0B0DF15C0813886
:100D700011F0813E89F491E090932438813E21F472
:100D800080913E38865F03C080913E388F5F8093AC
:100D90003E38BBDB8BE416DC80E008959C0190912B
:100DA0007338983088F4E92FF0E0EE0FFF1FEC580D
:100DB000F74C208331839F5F9093733848E0C901DB
:100DC0005BDF8091733808958FEF08950F931F9321
:100DD000CF93DF93EC018B0179DFB801CE01DF9176
:100DE000CF911F910F91DACF813C29F460E070E040
:100DF0008FE897E006C0823C39F460E070E085E55A
:100E000097E0E4DF80E0089581E00895843011F5F3
:100E100080918438909185382CE0833F920729F4A3
:100E200069E170E08AE798E013C08A57984061F45E
:100E300090916A38923040F0892F869596959695D4
:100E4000890FB5DC80E0089560E070E08FE897E0FE
:100E5000BDDFF8CF81E00895813C29F460E070E0C7
:100E60008FE897E006C0823C31F460E070E084EFE8
:100E700096E0ACDF16C0813B49F4CB016EE370E035
:100E80000E943312892B69F495DC0BC0813E59F422
:100E9000CB016EE370E00E9433126F5F60930C38F9
:100EA000C5DC80E0089581E00895CF93C0911A38A1
:100EB000C11117C0813C29F460E070E08FE897E031
:100EC00006C0823C31F460E070E085E797E07EDFA9
:100ED00009C0873B31F460E070E089E09BE05EDFB1
:100EE00001C0C1E08C2FCF910895813C29F460E0CE
:100EF00070E08FE897E006C0823C31F460E070E07B
:100F00008CE297E063DF07C0873B39F460E070E074
:100F10008DE09BE043DF80E0089581E00895CF936A
:100F2000DF93EB01883079F480E04CDB80910D3861
:100F3000837031DB10924538CD2B19F481E080931A
:100F40006B38C0E0D3C0813051F469317105C8F30A
:100F500080936B3880910D3883701DDBF2CF833026
:100F600029F580914B38882371F090914A3842ECF2
:100F700051E0949F9001959F300D112462177307E3
:100F800010F080931B386C2F80910D3811DE80910A
:100F900041388823B1F242EC51E0849F9001859F53
:100FA000300D11242C173D0760F64CC0813B91F4A5
:100FB00081E090E089DB06DB809147388111C1CF69
:100FC00080914838811103C0689708F4BACF61E076
:100FD00070E028C0813ED9F3813821F480911B381C
:100FE00090E013C0813C21F460916A3870E01AC02F
:100FF000823B79F48091193890911A38911180913F
:101000004938811104C086E990E05EDB05C086E9BD
:1010100003C0823E19F480E0D5DA93CF823C31F4EC
:1010200066E970E08AE798E0D1DE8BCF833999F3E7
:10103000833C29F460E070E085E597E0F5CF843CDF
:1010400031F4B8DB60E070E085E19BE0EDCF8D3BF3
:1010500049F4F89488ED84BF81E08093000178948E
:10106000A895FFCF8F3C29F460E070E082EF93E019
:10107000DBCF8A3B81F4CD2B19F5C0911A38CC23F4
:1010800021F098DB10921A3819C060E070E081E01E
:101090009BE084DE2BC0833B29F460E070E083EFAB
:1010A0009CE0C2CF873C61F490910D3881E0890FBC
:1010B00083709C7F982B90930D386DDAB7DB41CF0E
:1010C000C0911A38C11111C08A3C31F473DB81E040
:1010D00080931A38ABDB0AC0853C39F46BDB60E0E7
:1010E00070E08BE79EE072DE01C0C1E08C2FDF91E3
:1010F000CF9108959F92AF92BF92CF92DF92EF92DD
:10110000FF920F931F93CF93DF93182FEB01D09093
:101110001838F0901738A0904838AA2019F0B090ED
:10112000463802C0BB24B394C090193800911A38D5
:101130000111C0904938CC2051F041E0C41621F093
:1011400080911B388F1518F0A6E9EA2E01C0EF2C0C
:1011500090904538BE01812F3CDD209145382223F7
:1011600039F091100CC080916A388093283807C0FC
:10117000992029F060E070E08FE897E039C0812F76
:101180008D7F8830D9F4109240381A3019F4C0910C
:101190001B38D0E08D2D90E08C179D0738F48F2DF3
:1011A00090E0C817D90710F4C0931B38CE018CDA31
:1011B000FEDA81E08093053800E0D0C1113CD1F225
:1011C000123C71F480916A388E1510F48E2D02C095
:1011D00080911B38ECDA80916A3880932838ECCF04
:1011E000143C41F480E0EED960E070E085E19BE0E2
:1011F000EDDDE2CF8FE4810F823008F04FC0AA20EE
:1012000041F0CE0168E170E00E943312892B31F089
:10121000D3CF60910E3870E0CE01F6CF80916A385E
:10122000209761F4123B11F48FEF05C08F15E0F7A2
:10123000D81648F181E08093053825C020910E38FA
:1012400030E066E371E0269FA001279F500D369F96
:10125000500D11244C175D0710F48F1528F76CE61C
:1012600072E0269FA001279F500D369F500D11243C
:101270004C175D0740F4D81630F09CDA60E070E05F
:1012800085E19BE0A3DD3091053820916A384B2D34
:101290003403C0011124820F911D26C18FE1810FFB
:1012A000823020F480910538819584CF113009F087
:1012B000CFC0A99711F4109305382223B1F04091C3
:1012C000283830E021503109429FC001439F900DE2
:1012D00011246091443870E00E944712611101C0EE
:1012E00061E06093693860934C38C091693820910F
:1012F0006A388C2F90E0821B91096091263870919A
:1013000027386F5F7F4F6093263870932738009798
:1013100009F452CF97FF05C0233830F040E450E085
:1013200005C040E052E002C040E051E056954795CC
:1013300097FD0196959587950097C1F74617570732
:1013400008F03ACFC21710F48FEF03C02C1718F42F
:1013500081E0820F01C08C2F9FEF980F492F50E042
:10136000440F551FBA016F517D4FFB01A591B491F8
:10137000921770F420913A0A30913B0A232B41F4E2
:10138000AF3FB10529F4A0933A0AB0933B0A1FC0BE
:1013900020913A0A30913B0A2A173B0738F42091F2
:1013A0003A0A30913B0A2F5F3F4F0DC020913A0A15
:1013B00030913B0AA217B30750F420913A0A3091BA
:1013C0003B0A2150310920933A0A30933B0A9A0193
:1013D0002B543E4FF90145915491E091380AF09118
:1013E000390AE417F50738F44091380A5091390A60
:1013F0004F5F5F4F0DC0E091380AF091390A4E17E8
:101400005F0750F44091380A5091390A4150510910
:101410004093380A5093390AA0913A0AB0913B0A96
:10142000FB0145915491A417B50769F44091380A1E
:101430005091390AF901259134914217530719F453
:10144000C1D8C09369381092263810922738B4CE8C
:101450001530A9F480916A388B3508F4ADCE90E050
:101460008C1B9D0B282F8A3591052CF0873991050F
:1014700018F026E901C02AE5209369389DCE163080
:10148000B1F490916A3880914C38981708F094CE56
:10149000C90FD11D90E08C179D0734F0CA35D105D6
:1014A00024F4CAE5D0E001C0EC018C2F0EC0173047
:1014B00079F49091693880916A38891710F48F5FB8
:1014C00004C0981708F078CE81508093693874CEA4
:1014D000133C71F481E0A11080E080934838A6D9D4
:1014E00077D980916A3890E0EFD880931B3872CE1C
:1014F000011133C0133B49F4CD2B09F05DCECC2054
:1015000011F086E9E82E8E2D04C0133E21F480915F
:101510001B384DD923C0153C41F480E053D860E01E
:1015200070E08BE79EE052DC19C0173B29F460E0C5
:1015300070E08DEF9AE00FC01A3C39F480916A3860
:1015400080934B3873D936D909C01A3B31F460E027
:1015500070E085E09BE022DC01C001E0802FDF919C
:10156000CF911F910F91FF90EF90DF90CF90BF90A0
:10157000AF909F900895883061F41092253880E0F4
:1015800021D880916C38811136C081E08093253854
:1015900022C0982F907F903BB1F4209125384217BC
:1015A00078F0CB016DE570E05ED7029739F42F5FDC
:1015B000209325384217F8F088E303C082E101C088
:1015C00080E000D818C0903E61F4809125388823CF
:1015D00089F0481778F060E070E08FE896E0DEDB95
:1015E0000AC08A3041F460913E3880912538F90173
:1015F00009951CD96BDB80E0089529E233E043E0D4
:10160000BACF29E233E044E0B6CF24EC35E044E041
:10161000B2CF24EF33E041E0AECF28EF33E042E039
:10162000AACF23E134E041E0A6CF0F931F93CF93DD
:10163000DF93D82F8B0180798039B9F42091143849
:10164000909115388D2F8F70823041F480914B38F6
:10165000811108C0822F291728F403C0822F921706
:1016600008F4892F0E94E2021EC0803821F480E035
:101670000E94E20209C0D83039F480910D38869575
:1016800086950E94CB0254C0D13069F4093111050E
:1016900008F45AC0D0936B3880910D3886958695A2
:1016A0000E94CB0251C0D33039F480910D38602FA5
:1016B000869586957DDA48C0D33C31F47BD860E0CE
:1016C00070E08FE897E00AC0D43C89F4C0914B38B1
:1016D000CC2331F06C2F70E08AE798E077DB34C0E0
:1016E00060911B3870E08AE798E070DB30C0D43B33
:1016F00031F46ED81092C83861E070E0EDCFD53C7F
:1017000019F466E970E0E8CFD73C91F490910D3878
:10171000892F869586958F5F8370282F220F220F41
:101720009370920F90930D380E94CB027FD80CC01B
:10173000C0911A38C1110AC0DA3B41F460E070E090
:1017400081E19BE02BDB03C0C0E001C0C1E08C2F36
:10175000DF91CF911F910F910895CF93DF93C0E058
:10176000D6E08DE18E8385E58A83109293381092BE
:1017700094380E94A402E0EAF0E0808180618083D6
:1017800083E08883888581608887DF91CF91089581
:101790000F931F93CF9310926E388091C63890911B
:1017A000C7389C012F5F3F4F88279078822B932B5F
:1017B0008093C6389093C738C0916C380E94AD02B0
:1017C000C81731F110926B3880936C389091C838FB
:1017D000882359F0892F80699F709F3009F08F5FAF
:1017E0008093C83880E090E00DC0892F8F7E95FDF2
:1017F00002C0806801C0806C8093C8388091C63870
:101800009091C7380E9481021092C6381092C73852
:101810000091C6381091C73880916B38882379F0D1
:10182000B80183E00E9430020E944A020F73112720
:10183000012B09F043C010922A388FDF32C0C091CB
:10184000C8388C2F807F803B19F460E070E001C0C5
:10185000B80181E00E943002C4FF13C0C5FF02C07E
:10186000C8010CC008311105E0F01092C638109282
:10187000C738C062C093C83880E090E00E948102FF
:1018800010C0CC2371F0C5FD0AC00231110548F02B
:10189000C064C093C83880E090E00E9481020E943A
:1018A0008502C0912A38C11105C00E94A40281E0BE
:1018B00080938A38CF5FCF71C0932A38CF911F9120
:1018C0000F91089580919538811136D880916E38A6
:1018D00081115ECF0895EF92FF920F931F93CF93E4
:1018E000DF93EC010AEC18E082E3E82E82E0F82EA8
:1018F0002097D9F080914D38811119C080916A38B4
:10190000823028F485E00E942502C70104C081E0EE
:101910000E942502C8010197F1F781E00E9425028B
:10192000D1DF0E944A022197E3CF81E001C080E02D
:10193000DF91CF911F910F91FF90EF900895CF937A
:10194000C82F882391F089E10E94E20286EA90E0A4
:10195000C2DF80E00E94E2028AEF90E0BCDFC1506B
:1019600091F78AE992E0CF91B6CF89E10E94E20235
:1019700088E090E0B0DF80E00E94E2028AEF90E031
:10198000AADFEFCFCF93DF9364E661D5282F892FAD
:101990006AE05DD5EC01222341F0822FD0DF8C2F4D
:1019A000CEDF8D2FDF91CF91CACFC111F8CFF9CF04
:1019B000CF93DF93D82FC3E080911B380E94E202BF
:1019C00088EC90E088DFDD2319F080E991E083DF87
:1019D00080E00E94E20288EC90E07DDFC15061F778
:1019E000DF91CF910895DF92EF92FF920F931F93B3
:1019F000CF93DF93D82F8B01C0910B3881E0809378
:101A00004038C33009F0E2C0F09045388D2FE1D85E
:101A1000FF2051F080914538811106C060E070E0F0
:101A20008FE897E0D3D9D2C0D83021F481E08093F9
:101A30000338CEC0D23C19F410924538D7C0D13B00
:101A4000C1F490910238012B49F49E3610F08FEFCB
:101A500003C0923018F481E08093033880910338FA
:101A6000890F11F481E03CC18F3608F439C18EE64C
:101A700037C1D13E31F4809103388195809303388A
:101A8000ECC0D23B61F481E080930338809102384E
:101A9000823008F4EAC0815080930238E6C0D13029
:101AA00009F0F4C00932110511F4D0930338D09035
:101AB00023388D2D880FD7FC809527E0829FC001A9
:101AC0001124E09022382E2D220FE7FC2095D09192
:101AD00001382D9F90011124232F290FF0902138D8
:101AE0008F2D880FF7FC8095C09100388C9FC00126
:101AF0001124822F890F6091023870E0680F711DE8
:101B0000809145388130B9F48091423890914338C2
:101B100025E0969587952A95E1F724E730E0A9011D
:101B2000481B590B469FC001479F900D569F900D33
:101B30001124B90198D4862F0E94E20200FD06C04C
:101B40000E94B6028170D80ED0922338809120383E
:101B5000E80EE09222380E94B60265E278D4F90ECF
:101B6000F09221380E94B6028F7331F40E94B602BF
:101B70006DE06DD490932038DD2339F00E94B602D9
:101B80008F7319F4D150D09301380E94B60281119D
:101B900008C00E94B6026BE05AD4909301381092AC
:101BA0002238C33038F00E94B6028F7119F4C15048
:101BB000C09300380E94B6028F7709F07CC00E9463
:101BC000B60266E044D49093003875C0D83021F452
:101BD00081E08093043886C0D13C31F460E070E04D
:101BE0008FE897E0F3D87EC0D23C49F48C2F90E088
:101BF000019665E070E04BD480930B384CC0D13B2C
:101C000051F5C23090F400FD6DC0EC2FF0E0E75FBD
:101C1000F74C808190910438891B883020F08F3FE9
:101C200099F58EEF31C088E02FC0C43009F05AC05A
:101C30009091083880910438890F823010F482E046
:101C400003C0893708F088E7809308388091083806
:101C50000E94E20247C0D13E31F480910438819560
:101C60008093043818C0D23BA1F481E080930438FB
:101C7000C23068F500FD36C0EC2FF0E0E75FF74CAE
:101C800080818F3F79F18F5F80832CC0D13C09F434
:101C9000A5CFD23E19F40E94160424C0D53C39F4D5
:101CA00060E070E08BE79EE091D880E0D1CFD1304A
:101CB00011F081E018C00932110519F481E0809318
:101CC000043880916838080F009368380BC0C4301E
:101CD00049F480910838833008F4B8CF8150B4CFEC
:101CE0008093023880E0DF91CF911F910F91FF9098
:101CF000EF90DF9008950F931F93CF93DF93D82F2A
:101D00008B01883031F480914038813011F488E0C3
:101D10006ADE8D2F8079803961F481E080933F38CD
:101D2000C0914038C1110CC080911B380E94E20262
:101D300023C0803839F410923F3880E00E94E202DC
:101D4000C0E01AC0D130B9F4C0913F38CC2351F073
:101D5000809140388130A1F7B801DF91CF911F9178
:101D60000F9141CE0733114058F3D0936B3880E088
:101D70000E94CB0201C0C1E08C2FDF91CF911F9157
:101D80000F9108951F920F920FB60F9211242F9367
:101D90003F934F935F936F937F938F939F93AF93F3
:101DA000BF93EF93FF9381E080930B06809194386B
:101DB000882309F440C0E0919338E130D1F4809158
:101DC000211120912011A0911006B0911106A81B9D
:101DD000B10987FDB39530E06DD3DC01CB018058AC
:101DE0009F4FAF4FBF4F892F9A2FAB2FBB27BC01FF
:101DF00004C0609110067091110686E0660F771F8F
:101E00008A95E1F7F0E0EE0FFF1FDF01A157B74C15
:101E10006D937C93E557F74C8081918186179707E6
:101E200008F401966817790708F401978083918375
:101E300081E08093953881E080939438FF91EF9111
:101E4000BF91AF919F918F917F916F915F914F91D2
:101E50003F912F910F900FBE0F901F9018951F92DA
:101E60000F920FB60F9211248F9381E0809353014C
:101E700080936E388F910F900FBE0F901F90189522
:101E80001F920F920FB60F9211248F931D9A81E02B
:101E900080936D388F910F900FBE0F901F90189503
:101EA000F89480914000877F8093400088EDA8954A
:101EB00084BF90910001907F9093000121E030E079
:101EC00084BF2093610083E284B988E0809310048A
:101ED000809311048093120480931304809314045C
:101EE00099E09093150480931604809317048093CF
:101EF000320480933304809334048093500480939D
:101F00005104809352048093530487E38093010A21
:101F10008FEF90E08093360A9093370A91E0909388
:101F2000000A809112048160809312049093520100
:101F3000809151018111FCCF81E4809350010DDC2F
:101F4000789481E00E948F0260E070E086E097E084
:101F50000E94CE0610924D380E94DA030E94AD0214
:101F6000811108C0F89480E490E0B3D2853AA9F1D9
:101F70007894A9C0C0E08C2F0E94E20283E190E037
:101F8000AADC8C2F86950E94E20283E190E0A3DC1C
:101F90000E94AD028823B9F0CF5FC03461F7609131
:101FA000873880918638681B81E00E94F8030E9480
:101FB0001604C6E98C2F0E94E20284E090E08BDCDC
:101FC000C150C1F7CFCFCC2369F28C2F0E94E2021F
:101FD0008DE090E080DCC150F6CF0EE418E3C1E460
:101FE000D0E0CE0176D2F80181938F012196CB35D6
:101FF000D105B9F7789480914E3880934838809114
:102000004F388093143880915038809311388091E4
:10201000513880930E3880915238809315388091D2
:102020005338809312388091543880930F388091C0
:1020300055388093163880915638809313388091A4
:102040005738809310388091583880931A3880918F
:1020500059388093493880915A3880934738809115
:102060005B388093193880915C3880934B3880912D
:102070005D3880934A3880915E3880930B38809128
:102080005F38809309388091603880930A38809156
:102090006138809308388091623880930C38809141
:1020A000633880931C38809164388093863880919F
:1020B000653880931D388091663880930D38809103
:1020C00067388093413880914B38811180931B3859
:1020D00061E070E08FE897E00E94CE0644244394CC
:1020E0005524539447E0242ECC24C394D12C65E08E
:1020F000362E7CEF672E73E0772EE8EE8E2EE3E02F
:102100009E2EFFE8AF2EF7E0BF2E0E944A0280917C
:10211000713890917238009751F060916F387091DA
:1021200070380E94E60610927138109272388091D1
:102130006B38882309F45EC080E00E94E20240927E
:102140005201809151018111FCCFF9E5F0935001CA
:10215000809100068E7F809300060E94AD0281115F
:10216000FCCF0E948502809112048160809312044A
:102170001092953810926E3810926D3880916B38AD
:10218000882331F180915000897F846080935000D2
:10219000809150008160809350008895809150001C
:1021A0008E7F8093500080916D38811110926B3832
:1021B00080919538882331F050921E3850928A3899
:1021C0000E949C0480916E388823C1F2E1DAD6CF58
:1021D00022E020931E3880911204887F809312049D
:1021E000BCDA40925201809151018111FCCF31E45F
:1021F0003093500167DB10924D3880918438909174
:102200008538E3E0823F9E0779F4CCE7D0E0FE0119
:102210008491805394DB8CE291E05DDB2196F0E0C9
:10222000C838DF07A1F7C6C02CE0833F920779F0DA
:102230003EE08B37930709F0B2C08091403881307F
:1022400009F0F4C080913F38882309F4EFC0C091B1
:102250000B38C23011F120F0C43009F483C055CFDF
:10226000EC2FF0E0E75FF74CD08186E90E94E202B4
:10227000C11109C0DA3220F4C3010197F1F707C098
:1022800081E090E003C08D2F869590E024DB80E014
:102290000E94E2028D2F90E0C7C00E94B6028F73A9
:1022A000E82EF12C0E94B602622DD1D0E60102C0C8
:1022B000CC0FDD1F9A95E2F70E94B602632DC7D0BE
:1022C000F60102C0EE0FFF1F9A95E2F7CE0FDF1F57
:1022D0000E94B60290E0BE01DAD0C80FD91FC739FC
:1022E000D10514F0C6E9D0E08C2F0E94E202C701AC
:1022F000F2DA8E0133E0159507953A95E1F7011171
:1023000001C001E010E0C701E6DAC01BD10BD7FF26
:1023100002C0C0E0D0E08C2F0E94E2020E94B60210
:10232000837039F4C701D7DACE01959587950E945D
:10233000E202C230D1053CF70E94B6026DE087D0C0
:10234000E60102C0CC0FDD1F9A95E2F70E94B602AB
:1023500090E0BE0188D0C80FD91F80E00E94E20241
:10236000CE0162C0C0910838CC0FC73908F0C6E969
:10237000D4E08C2F0E94E20285E090E0ACDA8091FC
:1023800008380E94E20281E490E0A5DAD15089F792
:1023900080ED92E0A0DA80E00E94E202B6CEF7E0A3
:1023A00085359F0781F480918938ECDA80911A385D
:1023B000882381F0A0927138B092723810926F38F1
:1023C00010927038A2CE27E08537920731F48091C1
:1023D0008738D8DA88EE93E027C037E08C3293074D
:1023E000C1F480916C38811190CE80911B380E948D
:1023F000E20284E690E06FDA80E00E94E20220913F
:102400000C38289DC001299D900D112484569109F6
:102410000BC0845F964051F480E0CADA81E0C8DAEC
:1024200080E0C6DA80ED97E056DA6FCE80915000FA
:10243000897F80935000809150008160809350008C
:102440008895809150008E7F809350005ECE991BBE
:1024500079E004C0991F961708F0961B881F7A959B
:10246000C9F780950895AA1BBB1B51E107C0AA1F9D
:10247000BB1FA617B70710F0A61BB70B881F991F25
:102480005A95A9F780959095BC01CD01089597FBC9
:10249000072E16F4009406D077FD08D0E4DF07FC81
:1024A00005D03EF4909581959F4F08957095619564
:1024B0007F4F0895A29FB001B39FC001A39F700DED
:1024C000811D1124911DB29F700D811D1124911D3C
:1024D000089503D0808199270895FC01E050FC4EB7
:1024E0000895262FFADF0080021611F004D001971C
:1024F00001970895262FAF93BF93E0E0F0E132817A
:1025000031FDFDCFDC01A050BC4E2C932DE924BF42
:1025100023E020830196BF91AF910895F894FFCFF7
:10252000143811380E3800010201000000000000CC
:06253000010000000000A4
:10253600060B1801010100045A294303020D010785
:1025460005787890010A0A780101015A2D070200E0
:00000001FF
